:100000003428FF3FFF3FFF3F03138312A0018118F5
:100010000728811C092807130430A0002118142880
:100020008118102807131728811814280717A10C06
:1000300021181E28811C1A2807132128811C1E281C
:100040000717A10CA00B0E288118242807170800F9
:10005000993003138312A10004202208A100042078
:100060006430A10004200800031383129F010730AD
:1000700083169F00831285018316850183128601F2
:10008000FF3083168600831287010F3083168700A6
:100090008B0104308100831290011F30A3002330B4
:1000A000A4002830A5002D30A6003230A70037303C
:1000B000A8003C30A9004130AA004130AB004130DB
:1000C000AC00C830AD00C830AE00C830AF00C8309A
:1000D000B000C830B100C830B200C830B300C8307A
:1000E000B400C830B500C830B600870107178101D9
:1000F0000B112D08003A031DA62801300605F1005A
:100100007108003A031DA6281530AD00013007051F
:10011000F1007108003A031D8E28A30300308718F0
:100120000130F1007108003A031D9728A30A1E3020
:10013000230203189D281E30A3002308623C0318E5
:10014000A3286230A3002308A20028202E08003A2A
:10015000031DD428003086180130F1007108003AE0
:10016000031DD4281530AE0001300705F1007108D9
:10017000003A031DBC28A403003087180130F100A9
:100180007108003A031DC528A40A1E302402031872
:10019000CB281E30A4002408623C0318D12862300A
:1001A000A4002408A20028202F08003A031D0229D9
:1001B000003006190130F1007108003A031D0229D0
:1001C0001530AF0001300705F1007108003A031D3A
:1001D000EA28A503003087180130F1007108003AC1
:1001E000031DF328A50A1E3025020318F9281E3026
:1001F000A5002508623C0318FF286230A5002508E9
:10020000A20028203008003A031D3029003086194A
:100210000130F1007108003A031D30291530B0009B
:1002200001300705F1007108003A031D1829A603E3
:10023000003087180130F1007108003A031D2129B0
:10024000A60A1E302602031827291E30A6002608FB
:10025000623C03182D296230A6002608A20028203F
:100260003108003A031D5E290030061A0130F10002
:100270007108003A031D5E291530B10001300705F1
:10028000F1007108003A031D4629A70300308718C2
:100290000130F1007108003A031D4F29A70A1E30F2
:1002A0002702031855291E30A7002708623C0318AF
:1002B0005B296230A7002708A20028203208003AF4
:1002C000031D8C290030861A0130F1007108003AB4
:1002D000031D8C291530B20001300705F1007108AB
:1002E000003A031D7429A803003087180130F1007B
:1002F0007108003A031D7D29A80A1E302802031840
:1003000083291E30A8002808623C0318892962301E
:10031000A8002808A20028203308003A031DBA29A3
:100320000030061B0130F1007108003A031DBA29A4
:100330001530B30001300705F1007108003A031DC4
:10034000A229A903003087180130F1007108003A92
:10035000031DAB29A90A1E3029020318B1291E303A
:10036000A9002908623C0318B7296230A9002908AE
:10037000A20028203408003A031DE8290030861B1B
:100380000130F1007108003A031DE8291530B4006E
:1003900001300705F1007108003A031DD029AA03B6
:1003A000003087180130F1007108003A031DD92987
:1003B000AA0A1E302A020318DF291E30AA002A08C2
:1003C000623C0318E5296230AA002A08A20028200E
:1003D0003508003A031D162A003007190130F100D4
:1003E0007108003A031D162A1530B50001300705C3
:1003F000F1007108003A031DFE29AB030030871895
:100400000130F1007108003A031D072AAB0A1E30C3
:100410002B0203180D2A1E30AB002B08623C031878
:10042000132A6230AB002B08A20028203608003ABD
:10043000031D442A003087190130F1007108003A89
:10044000031D442A1530B60001300705F10071087C
:10045000003A031D2C2AAC03003087180130F1004C
:100460007108003A031D352AAC0A1E302C0203180D
:100470003B2A1E30AC002C08623C0318412A623033
:10048000AC002C08A200282000300B190130F1002C
:100490007108013A031D152B0B1187122D08003C22
:1004A0000318612AAD032D08003A031D602A0130AC
:1004B0000605F1007108003A031D602A0530AD0001
:1004C00087162E08003C0318752AAE032E08003A42
:1004D000031D742A003086180130F1007108003ABB
:1004E000031D742A0530AE0087162F08003C031840
:1004F000892AAF032F08003A031D882A0030061905
:100500000130F1007108003A031D882A0530AF0060
:1005100087163008003C03189D2AB0033008003AC3
:10052000031D9C2A003086190130F1007108003A41
:10053000031D9C2A0530B00087163108003C0318C3
:10054000B12AB1033108003A031DB02A0030061A5F
:100550000130F1007108003A031DB02A0530B100E6
:1005600087163208003C0318C52AB2033208003A45
:10057000031DC42A0030861A0130F1007108003AC8
:10058000031DC42A0530B20087163308003C031847
:10059000D92AB3033308003A031DD82A0030061BBA
:1005A0000130F1007108003A031DD82A0530B3006C
:1005B00087163408003C0318ED2AB4033408003AC7
:1005C000031DEC2A0030861B0130F1007108003A4F
:1005D000031DEC2A0530B40087163508003C0318CB
:1005E000012BB5033508003A031D002B0030071915
:1005F0000130F1007108003A031D002B0530B500F1
:1006000087163608003C0318152BB6033608003A47
:10061000031D142B003087190130F1007108003AD6
:10062000031D142B0530B60087167928162BFF3FC3
:02400E00723FFF
:00000001FF
